:10000000073099008122FE2A8B13C100030EC20023
:100010000A08C3006F228516C401051C4414851C00
:10002000C414441814281B28851CC414051C142847
:10003000851C14282228051C4414851C1B28051C1B
:100040001B282228440800380319382805192B28B2
:100050000330C4072B2885126F2285164F20051CFC
:1000600033288518382885126F2285166F222F288D
:1000700085120B1043088A00420E8300C10E410E08
:100080008B170900820744343734433446344734ED
:1000900052342034763431342E3434340034AD22AA
:1000A000C40303196928C40303196728C403031987
:1000B0006528C40303196328C403031961286B303E
:1000C0006B2857306B2843306B282F306B281B3040
:1000D0006B2807306B28D000C50079208520B1201F
:1000E000C320CD20DB20FB202921362240224F22B5
:1000F000080003309F2203309F2254309F22433058
:100100009F22B52231309F225A2A4D309F225930EA
:100110009F2243309F22B5220130C8000630C7001D
:100120004808E722C600203A0319982846089F226B
:10013000C80AC703031D90285008E722C6000F39DC
:1001400000380319592AB12246080F397522402375
:100150003B08303A0319AE283B089F223C089F22F7
:10016000592A50309F224F309F2253309F224330D4
:100170009F22B5225008E722C60007397522402386
:100180003C089F225A2A47309F2255309F22B52291
:100190003030C61931309F225A2A54309F225830AD
:1001A0009F2249309F22B522460E073975224023EF
:1001B0003C089F225A2A49309F2243309F224F30C9
:1001C0009F22B522C61FF12831309F222C309F225A
:1001D000D00A5008E722C6002F30C61B5C309F2291
:1001E000F62830309F222C309F22D00A5008E72278
:1001F0007F399F22592A5008E722C600C61F2629A8
:100200004D309F2250309F22B5225D220630B5002E
:100210003C3040233730840000089F220408840AC1
:100220003E3A031D0C29D00A5008E722C6005D2281
:100230000730B5003C3040233630840000089F2250
:100240000408840A3E3A031D1E29592A0630D007A5
:1002500008005008E722C6000B30C7004810C8103D
:1002600050309F2250309F22B5224508E722803926
:100270000319492952309F2245309F224C309F223A
:1002800041309F2259309F224608203A03195A2AAA
:10029000B3224608203A03195A2AC61B5329460896
:1002A0009F22C8141D2AC61346087839031D6D29DC
:1002B00057309F2249309F2244309F2245309F2251
:1002C0004608073903196B29752240233C089F22F1
:1002D000B1223C089F2248141D2A46087039031D8C
:1002E000882954309F2252309F2241309F22433030
:1002F0009F2245309F224608073903198629752217
:1003000040233C089F22B1223C089F2248141D2A0A
:1003100046086039031D9A2946080F397522402383
:100320003B08303A031996293B089F223C089F223C
:1003300048141D2A46085039031DA9294F309F2211
:100340004B309F2246080739752240233C089F22E4
:100350001D2A46084039031DB8294F309F224530D9
:100360009F2246080739752240233C089F221D2AF8
:1003700046083039031DC7294F309F224D309F2238
:1003800046080739752240233C089F221D2A46084B
:100390002039031DDA29B12246080F39752240237E
:1003A0003B08303A0319D6293B089F223C089F227C
:1003B00048141D2A46081039031D1D2A46080F3906
:1003C000031DEC2945309F2243309F2248309F2255
:1003D0004F309F2248141D2A46080E39031DFE295E
:1003E0004E309F224F309F2247309F2241309F2224
:1003F00054309F2245309F2248141D2A46080D394B
:10040000031D0C2A47309F2241309F2254309F22E7
:1004100045309F2248141D2A46080C39031D1C2A0A
:1004200049309F2247309F2241309F2254309F22E3
:1004300045309F2248141D2A1D2AC70303195A2A32
:10044000D00A5008E722C600203A03195A2AC81CCD
:10045000312AC61F332A460E0739053C0319332AB1
:10046000322A4818B3224810C8104D2944309F2220
:1004700054309F2258309F22B52232309F225A2A70
:1004800042309F2243309F224E309F22B5224508A2
:10049000E722C6003030461B31309F225A2A5430A2
:1004A0009F224E309F2243309F22B52231309F221F
:1004B0005A2AD00AAD226F2208003030BE00BD009B
:1004C000461BBE0A1F30C6054608A700D00A5008C2
:1004D000E722A600D00A5008E722A5000800000085
:1004E000C00B6F2ABF0B6F2A0800A500A701A60149
:1004F0000230B5003C300800CA000000CA0B7E2A5A
:10050000080083169F01FF239000051285129501B4
:100510001514951415158113161496148B15831242
:10052000051285120030E722C900D722CF00AF2282
:10053000AD220B1085166F2285128B170800CC0098
:100540000A30CB0003100512031C051649087C2253
:100550000314CC0CCB0BA32A08000D309F2A0A30C1
:100560009F2A2D309F2A2C309F2A20309F2A4C1002
:10057000851D00340930CB004F087C220310851DF7
:100580000314CC0C49087C220000CB0BBE2A4C087B
:10059000D101D201D10A0319D20A031963008519C6
:1005A000CA2A4C140800B7224C1CD32A0800CD00DC
:1005B000CE010310CD0C4D080319E52ACE07CD0C52
:1005C0004D080319E52ACE02D92A4E0808007F39C2
:1005D00083169B001C141A08831208007F398316A7
:1005E0009B008B131C1555309D00AA309D009C1458
:1005F0001C118B179C18FA2A83120800B7224C1C76
:10060000C8001B3A0319052BFE2AD322C8001B3A47
:100610000319052B4808443A0319172B4808553A83
:100620000319252B4808563A03193223FE2A8B1347
:10063000C801C80AD32283169A0083124808EE2202
:10064000C80AC81F1A2B8B17FE2A8B137F309F22D4
:10065000C801C80A4808E7229F22C80AC81F2A2BD7
:100660008B17FE2A8B13C801480842200038031953
:100670003C2B9F22C80A342BAD22AF228B170800D7
:100680008400AE010A30AD004D23220880003030D6
:1006900080078403B50B412B0800A301A201B3011D
:1006A000270DA20D2D08A2022E08031C2E0FA30257
:1006B0000301031C0130B302A70D0730B400270D5E
:1006C000A20DA30DB30D2D08271C702BA2022E081E
:1006D000031C2E0FA3020301031C0130B302792B6C
:1006E000A2072E0803182E0FA307030103180130D9
:1006F000B307A70DB40B5F2B260DA20DA30DB30DF1
:100700002D08271C8D2BA2022E08031C2E0FA302DE
:100710000301031C0130B302962BA2072E08031815
:100720002E0FA307030103180130B307A60D0730EE
:10073000B400260DA20DA30DB30D2D08261CAA2B67
:10074000A2022E08031C2E0FA3020301031C01307A
:10075000B302B32BA2072E0803182E0FA307030121
:1007600003180130B307A60DB40B992B250DA20D6C
:10077000A30DB30D2D08261CC72BA2022E08031CA7
:100780002E0FA3020301031C0130B302D02BA207DA
:100790002E0803182E0FA307030103180130B30717
:1007A000A50D0730B400250DA20DA30DB30D2D0826
:1007B000251CE42BA2022E08031C2E0FA30203010A
:1007C000031C0130B302ED2BA2072E0803182E0FD5
:1007D000A307030103180130B307A50DB40BD32BF6
:1007E0002518F82B2D08A2072E0803182E0FA30793
:0207F0000034D3
:02400E0084111B
:104200001E004F004B003100560043004600CE0018
:10421000490031008700A2003C0002002D00A400EC
:10422000C3004F004D0058008B008200200020008A
:104230002000200020000000700030008700A30054
:10424000160002002D00DE00A1004F004D005800B6
:10425000D20080008800E200E30087008F00890020
:10426000D9006200C700A2003C0042002D00A4005B
:104270008A002000200020002000200020002000D4
:104280002000200020000400E200EA0020002000BE
:10429000200020002000200020002000200020001E
:1042A0002000200020002000200020002000C50069
:1042B0000B003800200020002000200020002000FB
:1042C000B5004F004D005800D600E100E00020008E
:1042D00020002000200006007000450087008900B3
:1042E000870002002D0061009B00200020002000BC
:1042F00020002000200020002000200020000000DE
:00000001FF
